:1000000066C0000080C0000077C500007CC0000012
:100010007AC0000078C0000076C0000074C0000004
:1000200072C0000070C000006EC000006CC600000E
:100030006AC0000068C0000071C1000064C0000018
:1000400062C0000060C000000C9490090C94BF09CD
:100050005AC0000058C0000056C0000054C0000044
:1000600052C0000050C0000027675081C20D2E2DE5
:1000700007D3913D04320000060021656A55E43043
:1000800023B900070018146C070090876BF856110D
:10009000E92A001F4100072E050DD391FF08050036
:1000A000000C0021656A2D3B1322F862073F181DE2
:1000B0001CC700B0876BF8B611EA2A001F41002068
:1000C0002F2000203D2000424F56460D0A001124EB
:1000D0001FBECFEFD8E0DEBFCDBF11E0A0E0B1E0A2
:1000E000ECEBF4E102C005900D92A430B107D9F712
:1000F00011E0A4E0B1E001C01D92A73AB107E1F719
:1001000004D00C945C0A7CCF089584B7877F84BFA9
:1001100088E10FB6F89480936000109260000FBEE3
:10012000569A5E9A0E94F00980E091E060D284D2F3
:1001300082E08093030199EF97BD94E095BD84BD63
:1001400080936E00109280008AE08093810020E00E
:1001500030E080E80FB6F89480936100209361004E
:100160000FBE87E690E80E946B099FD281E08093E2
:1001700006015E98789484E890E09093570180930C
:10018000560181E00E945C090E947C092AD6EBD0CE
:1001900080916001882311F00E9410090E94820959
:1001A000F3CF8EBD0DB407FEFDCF8EB508955D98DB
:1001B000806C8EBD0DB407FEFDCF8EB51EBC0DB498
:1001C00007FEFDCF8EB55D9A08955D988EBD0DB486
:1001D00007FEFDCF8EB55D9A08951F931FEF84E350
:1001E000F4DF8AE090E0E8D01150C9F7E99A1F9156
:1001F00008951F93CF93DF93182F8B3010F018E0E2
:1002000002C0863008F015508BE290E0E12FF0E05C
:10021000E859FF4F1491EC012196CD3211F060E0C6
:1002200001C0612FBDD1C333D10511F0CE01F3CF91
:10023000DF91CF911F910895CF93DF9382E090E0FB
:10024000EC012196FE01E659FF4F6491A9D1CB3212
:10025000D10511F0CE01F4CF87E390E0EC012196B7
:10026000FE01E25AFF4F64919BD1C036D10511F0D7
:10027000CE01F4CF88E0BDDFDF91CF9108950F93D9
:100280001F93CF93DF938C01E998559A5D9A8EE185
:1002900090E092D05D988EE190E08ED05D9A8DE2F4
:1002A00090E08AD080E391DF84E690E085D05D988D
:1002B00080E48EBD0DB407FEFDCF8EB5C0E0D0E06A
:1002C000C8018C0F9D1F6AD18EBD0DB407FEFDCFF6
:1002D0008EB52196C932D10599F75D9A5D988EE762
:1002E0008EBD0DB407FEFDCF8EB58BE290E0EC0124
:1002F000219654D18EBD0DB407FEFDCF8EB5C3330C
:10030000D10511F0CE01F3CF5D9A83E35EDF81E08A
:1003100058D0DF91CF911F910F9108951F920F92A6
:100320000FB60F9211248F939F93AF93BF93809139
:10033000590190915A01A0915B01B0915C01019625
:10034000A11DB11D8093590190935A01A0935B01A7
:10035000B0935C01BF91AF919F918F910F900FBEB1
:100360000F901F9018958091590190910501891760
:1003700011F180930501A89580910401982F9F5F4A
:10038000909304018D37B8F010920401809103011D
:1003900081FF04C08BB190E489278BB980915D0106
:1003A00090915E0123E08438920728F4019690939F
:1003B0005E0180935D010895880F991F0197F1F701
:1003C000089520ED37E004C0F9013197F1F781502D
:1003D0008823D1F708951F93182F8091060180FF7D
:1003E0000CC080916301803208F08CD781E691E0E7
:1003F000612F35D11A3009F485D71F9108958DE00A
:10040000EADF8AE0E8CFCF93DF93EC0102C0E3DFBD
:100410002196FE0184918823D1F7DF91CF91089531
:10042000CF93DF93EC0102C02196D5DF888188232A
:10043000D9F7DF91CF910895A5E0B0E0E1E2F2E0D5
:10044000FEC71D82FE01349624E0382F3F702150F4
:100450003A3010F4305D01C0395C308334E0969559
:1004600087953A95E1F761503197009771F7822FA0
:100470008150992787FD9095FE013196E80FF91F6D
:1004800003C0215040833197615067FD02C01216AE
:10049000C4F3332727FD3095CE010196820F931FB9
:1004A000BFDF2596E2E0E7C790E062E040E3C4CF1B
:1004B000A6E0B0E0EDE5F2E0C0C7FC01262F1E8209
:1004C0008E010B5F1F4F35E03150CF016AE070E0C5
:1004D00092D7805DD8018C93CF016AE070E08BD712
:1004E000E62FF72F2150309751F4832F8150992711
:1004F00087FD9095FE013196E80FF91F08C0015065
:100500001040332309F7F1CF315040833197215008
:1005100027FD02C01316C4F3832F992787FD9095FA
:100520009E012F5F3F4F820F931F7ADF2696E4E0F4
:10053000A0C7FC01CB0125C0A32FA053AA3010F007
:10054000A0E002C02A2BA1E0B32FB154B63020F4B2
:10055000A32FA7532A2BA1E0B32FB156B63018F41E
:100560003755232B07C0AA2329F4303281F03A33C0
:1005700089F40DC0552341F0DB012D93BD0141509D
:1005800049F050E020E003C02295207F51E03191F6
:10059000332391F6681B790BCB01089577C7089533
:1005A0007DD7F999FECF0895A1E0B0E0E9EDF2E042
:1005B00046C71982009731F00196BE016F5F7F4FE9
:1005C00041E0B7DF8981882321F083E390E061E097
:1005D000E7DF10926E0028E088E190E00FB6F89413
:1005E000A895809360000FBE20936000FFCFCF934B
:1005F000DF93EC0180E090E061E0D2DF81E090E009
:1006000063E2CEDF19DE80E690E060E0C9DF81E6DC
:1006100090E060E0C5DF83E390E060E0C1DF84E369
:1006200090E062E0BDDF8981883719F080E090E0DA
:10063000BBDFDF91CF91089580E090E0AFDF8130A4
:1006400029F481E090E0AADF833219F080E090E0A5
:10065000CEDF84E390E0A2DF809303010895FC01E4
:100660008281803270F48F5F82838081DF01A80FE6
:10067000B11D13966C9313978F5F8083803209F4BA
:1006800010820895FC018281882371F08150828359
:100690009181DF01A90FB11D13968C9113979F5F74
:1006A0009183903209F4118208953E9A46985398A6
:1006B000E9E6F0E080818460808382EC91E09093B1
:1006C0005E0180935D0110921B0110925801089504
:1006D000AF92BF92CF92DF92EF92FF921F93CF9390
:1006E000DF93FC0110923F01109232012181220F11
:1006F000220F220F8381281B295F1092330180E093
:1007000030E097E077E010E0A0E057E0C52ED12C74
:1007100041E0E42EF12C7CC0EF01C10FD11D4C81D2
:1007200050E0072E02C0559547950A94E2F7B42F82
:10073000B170772311F0715002C01F5F77E06B3406
:1007400059F4933049F43323B9F5BB2311F031E068
:100750005FC010923F011EC09F3F79F56634F1F4EF
:10076000C82FD0E0CD5CDE4F4881042E4295402555
:10077000042E46954695402550E04F5F5F4F5595B6
:10078000479541705070CB2FD0E04C175D0761F05A
:1007900030933F018093320180E054C0653411F002
:1007A0006B3411F4BB23A1F38F5FC82FD0E0CD5C75
:1007B000DE4F188297E02CC030E0BB2341F1663455
:1007C00061F4C82FD0E0CD5CDE4F5701092E02C086
:1007D000AA0CBB1C0A94E2F717C0653411F06B3405
:1007E000B1F4C82FD0E0CD5CDE4FA92EBB24A7FC0E
:1007F000B094A6014A195B095A01A70102C0440F2F
:10080000551FAA94E2F75A0148814A29488391501A
:10081000AF5F4A2F4150421708F47ECF30933F011B
:10082000809332012A1708F0B7CF653411F49F3F47
:1008300011F0332319F08F5F8093320180913201E0
:10084000811181E0DF91CF911F91FF90EF90DF90B8
:10085000CF90BF90AF900895FC019281A081B181AB
:10086000A90FB11D8C912381322F31503383222364
:1008700021F49F5F928397E0938390E002C0959567
:1008800087952A95E2F7817008958F929F92AF9293
:10089000BF92CF92DF92FF920F931F93DF93CF937C
:1008A00000D0CDB7DEB74C0100E010E0FF2471E0CE
:1008B000A72EB12CC62EDD240894C108D1081FC074
:1008C000C4014A836983C8DF4A8169818823A9F00A
:1008D000442359F0C601801B910B950102C0220FE1
:1008E000331F8A95E2F7C90107C0C501002E02C077
:1008F000880F991F0A94E2F7F82A0F5F1F4F061717
:10090000F8F28F2D0F900F90CF91DF911F910F91E3
:10091000FF90DF90CF90BF90AF909F908F90089501
:10092000A4E0B0E0E5E9F4E083C5FC0110923201F7
:10093000218130E0A3E0220F331FAA95E1F78381E4
:10094000281B31092E3331050CF460C01B8287E06F
:100950008C833496FA83E98310E000E07E010894EA
:10096000E11CF11C2FC0C12EDD24C70168E040E06E
:100970008CDF23E331E0C20ED31EF6018083B82E54
:100980000B2CB294B0240B2CB694B694B024C701AF
:1009900063DF2B2D30E02F5F3F4F3595279521707A
:1009A000307090E02817390731F4C70155DF912FD7
:1009B0009F5F882319F01093320128C0F6018081CF
:1009C0000827192F163078F210933201C70168E01A
:1009D00040E05BDFC82E182F012E12951025012E46
:1009E000169516951025C70137DF212F30E02F5FB0
:1009F0003F4F359527952170307090E028173907C3
:100A000029F480E00C1519F481E001C080E02496FF
:100A1000E9E02AC5FC01A181B0E050E02081CD01D0
:100A2000841B950B0B9687319105E0F430E070E064
:100A3000C901861B970B8C309105A4F4EFEF853F1D
:100A40009E0784F02A0F3B1F261B370B241B350BF8
:100A50002C3031053CF480E09FEF253F39071CF036
:100A600081E0089580E00895282F30E0C901880FC3
:100A7000991F820F931F860F911D959587959595C8
:100A800087950895FC01A181AC3098F010926F0019
:100A9000E0912F01F0E084E190E09F01289FF001B8
:100AA000299FF00D389FF00D1124E95FFE4F108251
:100AB0000895662391F08A0F911DDC0121E030E05A
:100AC000038002C0220F331F0A94E2F714968C9120
:100AD0001497822B14968C9314978381982F91509E
:100AE0009383882341F487E0838381818F5F8183AF
:100AF000E80FF11D148208951F920F920FB60F9206
:100B00001124CF92DF92FF920F931F932F933F9365
:100B10004F935F936F937F938F939F93AF93BF9305
:100B2000EF93FF93DF93CF930F92CDB7DEB7809112
:100B30006001882321F082E080936001CBC0809126
:100B400084009091850054E0969587955A95E1F739
:100B5000182FF0902F0184E1F89E6001112427E006
:100B600031E0C20ED31EF6018081843031F41E3292
:100B700008F4B0C01F3408F09CC04B990CC08430FE
:100B800039F4C60161E07EDF109285001092840086
:100B9000109351019FC000915101101B10935201FD
:100BA0001092850010928400843021F4C60160E028
:100BB00069DF90C092E096BB882371F4053608F097
:100BC00089C0153608F086C0F601008B118B81E0D4
:100BD000828382E080837EC0823009F03EC0C601FD
:100BE0004096602F412F16DFF6019281882379F01D
:100BF0008089602F998338DFF601808B8189612F8E
:100C000033DFF601818B99819F5F928363C09430BB
:100C100008F19C3058F0F6012189808990E0820F1C
:100C2000911D8536910514F084E002C083E0F60141
:100C30008083F601028B138B118287E083831482F9
:100C400080EA9FE0909389008093880082E08093FF
:100C50006F0040C0F6011082B1CFC6014296602FEE
:100C6000412FD8DE882379F0C60161E00BDFF60161
:100C70008289602FF9DEF601828B8389612FF4DE91
:100C8000F601838B27C0C6014096602F412FC2DE3C
:100C9000882379F0C60160E0F5DEF6018089602FD7
:100CA000E3DEF601808B8189612FDEDEF601818B28
:100CB00011C010926F00EF2DF0E084E190E09F01F1
:100CC000289FF001299FF00D389FF00D1124E95F56
:100CD000FE4F10820F90CF91DF91FF91EF91BF9166
:100CE000AF919F918F917F916F915F914F913F91C4
:100CF0002F911F910F91FF90DF90CF900F900FBE1B
:100D00000F901F9018951F920F920FB60F921124FB
:100D10002F933F934F935F936F937F938F939F9303
:100D2000AF93BF93EF93FF9310926F0080915F0199
:100D300083FF02C08EE24FDB80912F01282F30E02D
:100D4000E4E1F0E0AF01249FF001259FF00D349F16
:100D5000F00D1124E95FFE4F9081933018F09181DE
:100D6000923030F410926F00E4E1F0E0CF0113C054
:100D7000909131019130D1F480915F0182FF03C0E5
:100D800087EC90E040DB10926F00E0912F01F0E0E3
:100D900084E190E09F01289FF001299FF00D389F8A
:100DA000F00D1124E95FFE4F10820AC09F5F9093FF
:100DB00031018F5F80932F01823011F410922F0147
:100DC000FF91EF91BF91AF919F918F917F916F9123
:100DD0005F914F913F912F910F900FBE0F901F90F9
:100DE0001895A0E0B0E0E6EFF6E021C38091520153
:100DF0008823C1F080915F0183FF12C082E7EBDAA4
:100E000080915F0184FF03C080915101E4DA86E69E
:100E1000E2DA80915F0184FF03C080915201DBDA46
:100E20001092520180913101882309F4F5C15E9A34
:100E30009091300184E1989FE0011124C95FDE4F59
:100E4000CE0166E445DC882341F180913201815076
:100E500080933201982F26E007C09150E92FF0E0EF
:100E6000ED5CFE4F3081230F9923B9F7E82FF0E0B6
:100E7000ED5CFE4F3081231711F486E48FC09CE0B7
:100E800007C08150E82FF0E0ED5CFE4F2081920F0B
:100E90008823B9F7931709F4A0C1CE0165E418DCE3
:100EA000882309F49CC180913201815080933201E2
:100EB000893009F094C190E08150E82FF0E0ED5CBA
:100EC000FE4F208192278823B9F780913C01981723
:100ED00009F085C185E462C0E0913201E150E09300
:100EE000320140913F012E2F30E095E080E013C0A9
:100EF0002150A22FB0E0AD5CBE4F5C91652F629592
:100F00006F708627960F442311F0332319F05F701A
:100F10008527950F3F5F222359F7980F9295907F71
:100F2000982BF0E0E41BF109ED5CFE4F80819817EF
:100F300061F08B81982F9F5F9B83873009F067C199
:100F40001B8289818150898362C18BE427C08B8198
:100F5000843009F0CDC0CE0140966CE34EE15ADDFD
:100F6000882309F4C5C0C801609151014EE152DDEA
:100F7000682FCE0187DD8C81809333018D81809332
:100F800034018E81809335018F818093360188856D
:100F90008093370185E08093320182E530915F01D3
:100FA00030FFA6C031FF02C020E059C020914001AF
:100FB00040913201241789F590E00FC0692F70E04D
:100FC000592F5F5FDB01AF5BBE4FFB01ED5CFE4F56
:100FD0007C916081761719F4952F921778F3941706
:100FE000E1F4E0905901F0905A0100915B011091F9
:100FF0005C01A0904D01B0904E01C0904F01D09087
:101000005001EA18FB080C091D0956E2E516F10427
:101010000105110510F421E001C020E090E00BC0B3
:10102000692F70E0FB01EF5BFE4F6D5C7E4FDB01D3
:101030005C9150839F5F941798F390934001409187
:10104000590150915A0160915B0170915C0140938C
:101050004D0150934E0160934F01709350018435C0
:10106000C1F436FD16C0909135019B3409F440C09F
:10107000993609F43DC0933509F43AC09435C1F16D
:101080009D37B1F19E37A1F190913601907790375D
:1010900079F1222369F59FD980913F01882329F0B6
:1010A0008091320181508093320100E007C0E02F2F
:1010B000F0E0ED5CFE4F8081F7D90F5FE0913201E7
:1010C0000E17A8F380913F01882351F0F0E0ED5C0A
:1010D000FE4F808190E08F70907061E040E3ACD96A
:1010E00080915F0185FF03C084E361D8DDD987D992
:1010F00080915F0182FF60C080E76DD9888190E0B8
:1011000062E040E2D5D9888990E0F4E0880F991F29
:10111000FA95E1F765E040E2CBD9898990E0E4E017
:10112000880F991FEA95E1F765E040E2C1D98A8905
:1011300090E074E0880F991F7A95E1F765E040E24E
:10114000B7D98B8990E064E0880F991F6A95E1F721
:1011500065E040E2ADD98A8190E063E040E2A8D941
:10116000898190E063E040E2A3D99B8127E030E0F1
:10117000A901491B5109CA0162E040E299D980E204
:101180002AD980915F0185FF05C084E310D88CD9EE
:1011900080E221D98B81873019F089818F5F898323
:1011A00000E006C0FE01E00FF11D84817DD90F5FD4
:1011B00089810817B8F323D91882809131018150B1
:1011C00080933101809130018F5F809330018230B4
:1011D00011F4109230015E981FC084E5DFCECE017D
:1011E0009FDB882311F088E4D9CE8E010E5E1F4F5D
:1011F000C801609151014B890DDC682FCE0142DCA2
:10120000CE016BE465DA882309F493CE65CE89813B
:10121000843009F06DCF9BCECDB7DEB7EAE023C1B5
:10122000A0E2B0E0E5E1F9E004C18091600188232B
:1012300009F43FC08130A9F4909153018091590184
:101240009817B9F185E30E94D700813129F48AE328
:101250000E94E5000E94ED008091590180935301A6
:1012600028C08FE30E94D700F82E8FE18F15F0F091
:101270005D988FEF0E94D1008E010F5F1F4F6801B4
:10128000E02E06C080E00E94D100F60181936F013C
:101290008C2D8E198F15B0F35D9A04C0F8018191E1
:1012A0008F0199D8802F8E198F15C0F381E080931C
:1012B0006001A096E8E0D9C0882351F087E390E070
:1012C0000E943F010E94ED0081E08093600108953B
:1012D00010926001089597FF04C022E02093C0009F
:1012E0009F779093C5008093C40088E08093C100ED
:1012F00086E08093C2000895E0915601F091570175
:10130000099508958091C10085FD09C08091630110
:10131000882329F08091C10080628093C1000895E4
:101320001F920F920FB60F9211242F933F934F935A
:101330005F936F937F938F939F93AF93BF93EF933D
:10134000FF938BB190E489278BB96091C60080919F
:10135000C000887119F484E891E081D9FF91EF9180
:10136000BF91AF919F918F917F916F915F914F91BD
:101370003F912F910F900FBE0F901F9018951F92C5
:101380000F920FB60F9211242F933F934F935F93B9
:101390006F937F938F939F93AF93BF93EF93FF933D
:1013A00080916301882331F081E691E06BD98093CD
:1013B000C60005C08091C1008F7D8093C100FF9160
:1013C000EF91BF91AF919F918F917F916F915F91BD
:1013D0004F913F912F910F900FBE0F901F90189536
:1013E0002D9A84B18C6284B9249880E58CBD8DB52A
:1013F00081608DBD0895AA1BBB1B51E107C0AA1FC8
:10140000BB1FA617B70710F0A61BB70B881F991FA5
:101410005A95A9F780959095BC01CD0108952F921A
:101420003F924F925F926F927F928F929F92AF9274
:10143000BF92CF92DF92EF92FF920F931F93CF93C1
:10144000DF93CDB7DEB7CA1BDB0B0FB6F894DEBF58
:101450000FBECDBF09942A88398848885F846E847E
:101460007D848C849B84AA84B984C884DF80EE80C8
:10147000FD800C811B81AA81B981CE0FD11D0FB6D1
:10148000F894DEBF0FBECDBFED010895F999FECFF0
:1014900092BD81BDF89A992780B50895262FF999B4
:1014A000FECF1FBA92BD81BD20BD0FB6F894FA9A47
:0C14B000F99A0FBE01960895F894FFCF42
:0414BC00787800023A
:00000001FF
